S02000006F70656E626C745F6F6C696D65785F73746D3332703130332E7372656307
S3150800000000500020C9440008194500081945000891
S3150800001019450008194500081945000800000000A0
S31508000020000000000000000000000000194500085C
S315080000301945000800000000194500081945000880
S31508000040194500081945000819450008194500080A
S3150800005019450008194500081945000819450008FA
S3150800006019450008194500081945000819450008EA
S3150800007019450008194500081945000819450008DA
S3150800008019450008194500081945000819450008CA
S3150800009019450008194500081945000819450008BA
S315080000A019450008194500081945000819450008AA
S315080000B0194500081945000819450008194500089A
S315080000C0194500081945000819450008194500088A
S315080000D0194500081945000819450008194500087A
S315080000E019450008194500081945000800000000D0
S315080000F000000000000000000000000000000000F2
S3110800010000000000000000005FF808F195
S3150800010C10B5054C237833B9044B13B10448AFF337
S3150800011C00800123237010BDD401002000000000CC
S3150800012CD045000808B5034B1BB103490348AFF388
S3150800013C008008BD00000000D8010020D04500084A
S3150800014C72B6704762B67047F0B5002401E0013408
S3150800015CE4B2112C20D8114D15F8147005EB440592
S3150800016C95F801E007EB0E0505FB000548F6A04CD3
S3150800017C9CFBF5F605FB16C6002EE8D19CFBF5F59F
S3150800018CADB20D80013DADB2B5F5806FDFD21770FB
S3150800019C83F800E00120F0BD0020F0BD10460008F1
S315080001AC10B582B001AB0DF105020DF106014FF445
S315080001BCFA70FFF7C9FF012803D0F921464800F069
S315080001CCEBFC464B00225A611A6842F400421A604C
S315080001DC00F018FC00F1FA04404B1B6813F4004FAE
S315080001EC05D000F0AAFD00F00DFC8442F4D23B4B7E
S315080001FC1A6822F002021A601A6842F001021A60A2
S3150800020C00F000FC00F1FA04344B5B6813F0010FA4
S3150800021C05D100F092FD00F0F5FB8442F4D29DF86E
S3150800022C05305A1E9DF80430013B1B0543EA024370
S3150800023CBDF80620013A1343284AD361136823F004
S3150800024C0103136000F0DEFB00F1FA04234B5B6834
S3150800025C13F0010F05D000F070FD00F0D3FB8442BB
S3150800026CF4D21E4BD3F8002242F00102C3F8002246
S3150800027CD3F81C2222F00102C3F81C22D3F80C2254
S3150800028C42F00102C3F80C22D3F8042222F0010230
S3150800029CC3F80422124AC3F8402202F14C52043223
S315080002ACC3F84422D3F8042222F00102C3F804222C
S315080002BCD3F8142222F00102C3F81422D3F81C2214
S315080002CC42F00102C3F81C22D3F8002222F00102E4
S315080002DCC3F8002202B010BDE845000800640040CF
S315080002EC0000E0CC38B504460D46254B9B6813F048
S315080002FC806F3ED0224BD3F8802102F00102C3F85E
S3150800030C8021D3F8802142F07C4242F40012C3F8D3
S3150800031C8021C3F88451E178A278120442EA01627A
S3150800032C617842EA012221780A43C3F88821E179E7
S3150800033CA279120442EA0162617942EA0122217920
S3150800034C0A43C3F88C21D3F8802142F00102C3F882
S3150800035C802100F057FB00F13204094B9B6813F01F
S3150800036C806F05D100F0E9FC00F04CFB8442F4D216
S3150800037C38BD40F26311034800F00EFCBAE700BF23
S3150800038C00640040E8450008244BDB6813F0030FB3
S3150800039C41D0224BD3F8B03113F0040F0ED11F4BBA
S315080003ACD3F8B0315B0D40F2676293420DD0002052
S315080003BC1A4AD36843F02003D3607047174BD3F817
S315080003CCB031DB0843F00043EDE7144BD3F8B42106
S315080003DC02F00F020A70D3F8B8210270D3F8B821CC
S315080003EC120A4270D3F8B821120C8270D3F8B821CD
S315080003FC120EC270D3F8BC210271D3F8BC21120AB2
S3150800040C4271D3F8BC21120C8271D3F8BC311B0E85
S3150800041CC3710120CCE70020704700BF0064004080
S3150800042C08B5FFF78DFE08BD10B500F0AFFA00B998
S3150800043C10BD00F03FFC00F0BDFA00F0ABFA20F05E
S3150800044C604020F07F00044B186000F0A3FA446863
S3150800045CFFF778FEA047EBE708ED00E070B508E07B
S3150800046C461C4D1C0B78037000F067FC3046294679
S3150800047C2246531E9CB2002AF2D170BD044B054A83
S3150800048C5A6002F188325A603422DA60704700BF2B
S3150800049C0020024023016745024A136943F0800392
S315080004AC136170470020024038B50546002401E068
S315080004BC0134E4B20C2C15D800F03FFC04EB4402D2
S315080004CC9300094AD358AB42F2D804EB4402910084
S315080004DC054A0A44526813449D42E9D2024B0B441E
S315080004EC187A38BDFF2038BD3446000838B505469D
S315080004FC00240C2C10D800F020FC04EB44039A00C2
S3150800050C074B13441B7AAB4202D00134E4B2F0E732
S3150800051C1346034AD05838BD4FF0FF3038BD00BFDC
S3150800052C3446000838B5054600240C2C10D800F0C3
S3150800053C04FC04EB44039A00064B13441B7AAB42A7
S3150800054C02D00134E4B2F0E7024B1344586838BDC4
S3150800055C002038BD3446000808B5C1F3080353B962
S3150800056C0368994209D040F8041B4FF40072FFF750
S3150800057C75FF012008BD002008BD012008BD00003C
S3150800058C2DE9F84F81460068FFF78EFFFF2856D0F5
S3150800059CFFF774FF2B4BDB6813F0010F08D1294AC0
S315080005AC136943F00103136100254FF0010A09E0B2
S315080005BCFFF772FF4FF0000A3EE058F807309E42EC
S315080005CC31D101357F2D30D8D9F80080AF0008EB32
S315080005DC070B09EB07035E68B3B228F8253000F061
S315080005EC11FA441D174BDB6813F0010F07D000F006
S315080005FCA4FB00F007FA8442F4D24FF0000A330C3D
S3150800060CABF8023000F0FEF9441D0E4BDB6813F014
S3150800061C010FD2D000F091FB00F0F4F98442F4D229
S3150800062C4FF0000AC9E74FF0000A064A136923F08F
S3150800063C01031361FFF730FF5046BDE8F88F4FF002
S3150800064C000AF9E70020024038B50D460B4B9842D4
S3150800065C08D004460A4B994206D0FFF791FF20B9F9
S3150800066C002407E0074C00E0044C29462046FFF717
S3150800067C73FF08B1204638BD0024FBE7F4030020BD
S3150800068C00600008F00100202DE9F04106460C46F2
S3150800069C17461D4621F4FF7828F001080368B3F1C4
S315080006ACFF3F0DD03368984505D041463046FFF7D5
S315080006BCCBFF064628B33368E41A344404340CE0FA
S315080006CC4146FFF749FF03460028EBD116E017F819
S315080006DC013B04F8013B013D0FD000F02EFB331D06
S315080006ECE31AB3F5007FF2D308F500713046FFF72D
S315080006FCABFF064638B1041DE9E701231846BDE8E9
S3150800070CF0810023FAE70023F8E700002DE9F04111
S3150800071C884251D8022853D90F2901D900264CE012
S3150800072C0D460446FFF7AAFE264BDB6813F0010FAD
S3150800073C19D1244A136943F0020313612046FFF7C3
S3150800074CD5FE80462846FFF7D1FE07462846FFF712
S3150800075CE9FE0744013FA7EB08070137C7F38F27C4
S3150800076C0126002505E0FFF797FE002625E0013552
S3150800077CADB2BD4218D208EB8522124B5A611A69E2
S3150800078C42F040021A6100F03DF900F164040D4B89
S3150800079CDB6813F0010FEAD000F0CFFA00F032F95B
S315080007AC8442F4D20026E2E7064A136923F00203D0
S315080007BC1361FFF771FE00E000263046BDE8F081B4
S315080007CC0026FAE7002002404FF0FF33024A136076
S315080007DC024A1360704700BFF0010020F4030020A2
S315080007EC70B54B1E154C241AA34201D9002070BDB6
S315080007FC16460D460446FFF757FEFF281AD0281949
S3150800080C0138FFF751FEFF2816D024F4FF7323F0A6
S3150800081C01030B4A934206D02B4632462146094819
S3150800082CFFF732FF70BD2B46324621460648FFF7C6
S3150800083C2BFF70BD002070BD002070BDFFFF0108A6
S3150800084C00600008F0010020F40300204A1E0E4B3D
S3150800085C1B1A9A4201D90020704770B50C460546FA
S3150800086CFFF722FE064660190138FFF71DFEFF2E1C
S3150800087C06D0FF2806D001463046FFF747FF70BD65
S3150800088C002070BD002070BDFFFF0108104B1B68CF
S3150800089CB3F1FF3F1AD000B583B00D4A536891687F
S315080008AC0B44D1680B4411690B4451690B4491698B
S315080008BC0B44D26913445B4202AA42F8043D042154
S315080008CC0448FFF78DFF03B05DF804FB0120704761
S315080008DCF40300200C6100080D4B1B680D4A1268C6
S315080008EC13440D4A126813440C4A126813440C4AF2
S315080008FC126813440B4A126813440B4A12681344C1
S3150800090C0A4A1268D34201D000207047012070476A
S3150800091C0060000804600008086000080C60000805
S3150800092C1060000814600008186000080C610008C4
S3150800093C08B50C4B1B68B3F1FF3F04D00948FFF709
S3150800094C1FFE034650B1084B1B68B3F1FF3F07D097
S3150800095C0548FFF715FE034600B10123184608BDE6
S3150800096C0123FBE7F4030020F00100200048704740
S3150800097C0060000808B5FFF727FF08BD08B5FFF7A4
S3150800098C2FFF08BD08B5FFF761FF08BD08B5FFF7CF
S3150800099CA3FF08BD08B5FFF7E9FF08BD08B5FFF7C3
S315080009AC75FF034608B9184608BDFFF7C1FF03468D
S315080009BCF9E700000022014B1A60704710E000E0CE
S315080009CC08B5FFF7F7FF054B054A5A6000229A60EF
S315080009DC05211960034B1A6008BD00BF10E000E042
S315080009EC3F190100F8050020044B1B6813F4803FDF
S315080009FC03D0034A136801331360704710E000E014
S31508000A0CF805002008B5FFF7EFFF014B186808BD7D
S31508000A1CF8050020054B1B8813F0200F04D0034B58
S31508000A2C9B880370012070470020704700440040E3
S31508000A3C0E4B1B8813F0800F01D10020704710B5A0
S31508000A4C80B20A4B9880FFF7DDFF00F10A04074BCA
S31508000A5C1B8813F0800F07D100F06FF9FFF7D2FF50
S31508000A6C8442F4D2002010BD012010BD0044004081
S31508000A7C084B00221A819A811A829A821A8340F2AA
S31508000A8C71221A819A8992B242F4005242F00C02EF
S31508000A9C9A8170470044004070B506460D464029B9
S31508000AAC0AD82846FFF7C4FF012803D093210E481D
S31508000ABC00F072F8002406E08F210B4800F06CF861
S31508000ACCEFE70134A4B2ABB29C420BD200F035F975
S31508000ADC305DFFF7ADFF0128F3D09C21024800F0EA
S31508000AEC5BF8EEE770BD00BFD046000870B5254B25
S31508000AFC1C78BCB92448FFF78DFF012801D0204685
S31508000B0C70BD214B1B78013BDBB23F2BF7D8FFF7A7
S31508000B1C79FF1E4B186000221D4B1A700122194BC7
S31508000B2C1A70ECE706460D46194B1B780133164826
S31508000B3C1844FFF76FFF044601280AD0FFF762FF37
S31508000B4C124B1B686433984219D900240D4B1C7040
S31508000B5CD5E70F4B1A780132D2B21A700A4B1B78AA
S31508000B6C9A4201D00024CAE70A493046FFF776FCB8
S31508000B7C0022044B1A70064B1B782B70BFE7002417
S31508000B8CBDE700BF3D060020FC05002040060020FE
S31508000B9C3E060020FD05002008B500F0CEF8FCE75F
S31508000BAC08B500F0C5F8012806D000F051F918B1BF
S31508000BBC0B4B1B78012B00D008BDFFF723FF094B05
S31508000BCC1B6803F5FA739842F6D30022044B1A7085
S31508000BDC00F048F90028EFD1FFF726FCECE700BF38
S31508000BEC440600204806002008B50122044B1A705A
S31508000BFCFFF708FF034B1860FFF7D2FF08BD00BFCD
S31508000C0C440600204806002008B5FFF709FC00F04A
S31508000C1C93F8FFF7D5FEFFF7ADFE00F001F900F0EB
S31508000C2C0FF8FFF7E1FF08BD08B500F086F8FFF7E7
S31508000C3CDBFE00F025FA00F013F8FFF7B1FF08BD4C
S31508000C4C10B502F0B7FCFFF7ABFA044C012323707E
S31508000C5CFFF70EFF0023237010BD00BF0000002015
S31508000C6C00B583B00DF107011048FFF78DFB01287D
S31508000C7C09D00DF107010D48FFF738FF01280BD0F5
S31508000C8C03B05DF804FB0122094B1A709DF8071096
S31508000C9C064802F0AFFCECE70022054B1A709DF8EB
S31508000CAC0710024802F0A6FCEAE700BF4C06002033
S31508000CBC000000207047000038B504460D46094B65
S31508000CCC1B78012B05D0074B1B7833B102F08AFC35
S31508000CDC38BDC9B2FFF706FBF5E7E9B22046FFF7C0
S31508000CECDBFEF3E700000020074B1B78022B05D030
S31508000CFC032B05D0012B05D04020704700207047E8
S31508000D0C002070470820704700000020074B1B780E
S31508000D1C022B05D0032B05D0012B05D0402070479C
S31508000D2C00207047002070470820704700000020FC
S31508000D3C08B502F04DFC08BD7047704710B4034661
S31508000D4C01310C4AA2FB0323DB08F9D100230B70F3
S31508000D5C084BA3FB0023DB081A4603EB83035C0052
S31508000D6C031B303301F8013D1046002AF0D1084622
S31508000D7C10BC7047CDCCCCCC00F00F03092802D997
S31508000D8C03F13700704710B503F1300403F0E4FBA8
S31508000D9C2044437803F00303022B01D0E0B210BDC4
S31508000DAC203CFBE738B505460C460009FFF7E4FF7F
S31508000DBC207005F00F00FFF7DFFF60700023A370AB
S31508000DCC204638BDF8B5074600252E4607E0203CD8
S31508000DDC10E03301DBB21344DEB20135EDB2012D5E
S31508000DEC19D87C5D03F0B8FB2044437803F0030361
S31508000DFC022BECD0E3B2A3F13002D2B2162A09D8F0
S31508000E0CA3F13A01C9B2062907D9092AE1D9373B10
S31508000E1CDAB2DEE700263046F8BD0026FBE700000E
S31508000E2C08B50022064B1A700649074801F052FD10
S31508000E3C00B908BD77210548FFF7AEFEF9E700BFF4
S31508000E4CEC0A0020FC46000894060020004700081F
S31508000E5C034B1B780BB1002070470120704700BF6D
S31508000E6CEC0A002008B5FFF763FF01280ED0084BE3
S31508000E7C1B780BB1002008BD02F02EFC012801D00E
S31508000E8C002008BD0122024B1A7008BD002008BDBF
S31508000E9CEC0A002038B50546047803F05DFB2044BF
S31508000EAC437803F00303022B03D0532C03D00320FF
S31508000EBC38BD203CF9E703F04FFB6B7818444278B1
S31508000ECC12F0040F01D1032038BD312B07D0322B79
S31508000EDC07D0332B01D0032038BD022038BD0020A3
S31508000EEC38BD012038BD70B506460230FFF76AFFDB
S31508000EFC054684B204363046FFF764FF0544EDB266
S31508000F0C013CA4B20236012CF5D8ED43EDB23046BD
S31508000F1CFFF758FF854201D0002070BD012070BD37
S31508000F2C2DE9F041044616468846A1B198B12046EB
S31508000F3CFFF7B0FF0546032800F099802046FFF717
S31508000F4CD2FF002800F09780012D2DD04DB1022D2F
S31508000F5C57D000278CE040F261214848FFF71CFE69
S31508000F6CE5E7A01CFFF72EFF87B2201DFFF72AFF27
S31508000F7C0002C8F80000A01DFFF724FFD8F80030BF
S31508000F8C1844C8F800000834033F3FB2002E6FD04F
S31508000F9C002506E02046FFF715FF7055023401358B
S31508000FACADB2BD42F6DB63E0A01CFFF70BFF87B2C0
S31508000FBC201DFFF707FF0004C8F80000A01DFFF767
S31508000FCC01FFD8F8003003EB0020C8F8000004F144
S31508000FDC0800FFF7F7FED8F800301844C8F80000E8
S31508000FEC0A34043F3FB2002E42D0002506E02046C4
S31508000FFCFFF7E8FE705502340135ADB2BD42F6DB9B
S3150800100C36E0A01CFFF7DEFE87B2201DFFF7DAFEDE
S3150800101C0006C8F80000A01DFFF7D4FED8F800306B
S3150800102C03EB0040C8F8000004F10800FFF7CAFEFD
S3150800103CD8F8003003EB0020C8F8000004F10A00C9
S3150800104CFFF7C0FED8F800301844C8F800000C3476
S3150800105C053F3FB266B1002506E02046FFF7B2FE13
S3150800106C705502340135ADB2BD42F6DB00E00027FF
S3150800107C3846BDE8F0814FF0FF37F9E7004700081E
S3150800108C964B1B78002B00F0F18170B5012B05D01F
S3150800109C022B2DD0032B00F03F8170BDFFF76AFCA5
S315080010AC02F03CFB8E4802F07DFB8E4802F07AFB80
S315080010BC02F030FB012201468B4801F037FC30B1B7
S315080010CC8A4802F06FFB012002F05EFB70BD88486F
S315080010DC02F068FB874802F065FB874802F062FB62
S315080010EC864B00221A605A6002227C4B1A7070BD1D
S315080010FC834C04F50C724FF48071824802F030F878
S3150800110C94F84132002B5ED1002877D07D48002216
S3150800111C00F5C071FFF704FF0446B0F1FF3F60D03D
S3150800112C002C09DD754B5B68002B69D1754BD3F820
S3150800113C8021724B1A605C60714BD3F84422D3F849
S3150800114C3C329A42A9D10021674801F0C5FE002815
S3150800115C40F0A980694B5B6873B3654802F022FBC3
S3150800116C694802F01FFB694D644C29466068FFF715
S3150800117CE5FD284602F016FB654802F013FB2946E6
S3150800118CE078FFF70FFEA91CA078FFF70BFE291DC8
S3150800119C6078FFF707FEA91D2078FFF703FE28469F
S315080011AC02F000FB5B4802F0FDFA61682068FFF765
S315080011BCE9FB002800F084804D4802F0F3FA03227C
S315080011CC464B1A7070BD494802F0ECFA022002F040
S315080011DCDBFA04F50C7001F06BFE00223F4B1A701B
S315080011EC70BD424802F0DEFA032002F0CDFA3E4802
S315080011FC01F05EFE0022394B1A7070BD00248FE791
S3150800120C404AD2F880113D4A12681A44914239D0A4
S3150800121C374802F0C7FA3C4802F0C4FA3B4E374D41
S3150800122C31466868FFF78AFD304602F0BBFA384843
S3150800123C02F0B8FA3146E878FFF7B4FDB11CA87885
S3150800124CFFF7B0FD311D6878FFF7ACFDB11D2878A6
S3150800125CFFF7A8FD304602F0A5FA2E4802F0A2FACE
S3150800126C69682868FFF78EFB80B1214802F09AFA64
S3150800127C214802F097FA234BD3F880211F4B1A60AA
S3150800128C5C6059E723441D4A536055E7174802F03A
S3150800129C89FA052002F078FA134801F009FE0022B3
S315080012AC0E4B1A7070BD114802F07CFA042002F03D
S315080012BC6BFA0D4801F0FCFD0022084B1A7070BD44
S315080012CC0A4802F06FFA052002F05EFA064801F0A9
S315080012DCEFFD0022014B1A7070BD00BFEC0A00200E
S315080012EC1C47000840470008C40800206847000847
S315080012FC70470008784700089C4700088C060020B1
S3150800130C94060020F00A0020CC470008740C002034
S3150800131CD84700087C480008554C04F50C724FF465
S3150800132C8071544801F01CFF94F84132002B66D1A9
S3150800133C00287FD04F4800F5807200F5C071FFF782
S3150800134CEFFD0546B0F1FF3F67D0002D34DD4A4866
S3150800135C02F028FA494C21462846FFF7EFFC2046AE
S3150800136C02F020FA464802F01DFA424E214696F83B
S3150800137C8301FFF717FDA11C96F88201FFF712FDF2
S3150800138C211D96F88101FFF70DFDA11D96F8800128
S3150800139CFFF708FD204602F005FA3A4802F002FA71
S315080013AC06F580722946D6F88001FFF7E7FA002879
S315080013BC42D0354802F0F6F92D4BD3F84422D3F82F
S315080013CC3C329A427FF469AE304802F0EBF9FFF7EB
S315080013DCE5FA00283DD02C4802F0E4F92C4802F036
S315080013ECE1F92C4801F064FD2B4802F0DBF90022E8
S315080013FC2A4B1A7002F0A6F9FFF716F84DE628489C
S3150800140C02F0D0F9022002F0BFF904F50C7001F0D5
S3150800141C4FFD0022214B1A7070BD224802F0C2F90A
S3150800142C032002F0B1F91B4801F042FD00221B4BC8
S3150800143C1A7070BD002588E71B4802F0B3F9062020
S3150800144C02F0A2F9134801F033FD0022134B1A706F
S3150800145C70BD154802F0A6F9072002F095F90D485B
S3150800146C01F026FD00220D4B1A7070BD704700BFA7
S3150800147C94060020F00A00203C480008740C002052
S3150800148C4C4800087C480008704700086448000867
S3150800149C80480008C408002098480008EC0A002078
S315080014ACF44700081848000868470008427800788E
S315080014BC40EA02207047C278837843EA02224378CE
S315080014CC43EA0223007840EA032070470170090AB0
S315080014DC417070470170C1F307234370C1F307438A
S315080014EC8370090EC170704713462AB10A780270C8
S315080014FC01300131013BF9D1704701700130013AD5
S3150800150CFBD1704730B4451C037808781B1A013A8E
S3150800151C04D04C1C28462146002BF4D0184630BC67
S3150800152C704700E0013003780BB18B42FAD11846AC
S3150800153C704702394369023B994204D24389806A4F
S3150800154C03FB010070470020704770B506460D4630
S3150800155C01F11A00FFF7AAFF04463378032B00D0D3
S3150800156C70BD05F11400FFF7A1FF44EA0040F7E748
S3150800157C70B506460C46154691B204F11A00FFF7EB
S3150800158CA5FF3378032B00D070BD290C04F1140089
S3150800159CFFF79CFFF8E700002DE9F04180460F465F
S315080015AC01F11A00FFF782FF58BB3D7805F03F059D
S315080015BC013D05EB450305EB83050126002404E0F4
S315080015CC4FF6FF73984222D101340C2C0DD8144BCC
S315080015DC185D3844FFF76AFF002EF1D0FE2D13D89C
S315080015EC28F8150006460135EEE73B7813F0400F50
S315080015FC10D0FE2D11D8002328F815300120BDE88F
S3150800160CF0810020BDE8F0810020BDE8F0810020C3
S3150800161CBDE8F0810120BDE8F0810020BDE8F0812D
S3150800162C444900082DE9F84380460F4691464B730A
S3150800163C0F23CB7200240C73214607F11A00FFF70F
S3150800164C45FF09F1FF3606EB460306EB83062546EE
S3150800165C02E001340C2C11D84FF6FF739D4202D0D0
S3150800166C38F8165001360C4B185D29463844FFF7E6
S3150800167C2DFF002DEDD14FF6FF75EAE74FF6FF73F8
S3150800168C9D4202D038F816300BB949F0400987F854
S3150800169C0090BDE8F88300BF4449000870B582B0D5
S315080016AC054616461C460B22FFF71EFF052C11D8BD
S315080016BC07231FE001310F290DD802F0010000EBBA
S315080016CC4303520813F4803FF4D083F4883383F031
S315080016DC2103EFE72346328812B102360021EAE7E6
S315080016EC1C46E5E75A1E02A8034403F8081C2409FD
S315080016FC09D0134604F00F0202F130013929F1D949
S3150800170C02F13701EEE77E210346134403F8081C61
S3150800171C00E00134944208D22B5D202BF9D104E069
S3150800172C202018700C46072909D8611C2B19072A82
S3150800173CF6D802A8104410F8080C0132F1E702B0EA
S3150800174C70BD01460B220020C30143EA5003DBB2ED
S3150800175C08780344D8B20131013AF5D170470168CB
S3150800176C09B10A4603E04FF0FF3308E0013213785B
S3150800177C1F2B01D93A2BF9D13A2B02D00023184644
S3150800178C704710B44C1C0B78303B092B07D8A24277
S3150800179C08D153B901320260184610BC70474FF095
S315080017ACFF33F9E74FF0FF33F6E74FF0FF33F3E774
S315080017BC38B50C4620B1054603680BB11A781AB928
S315080017CC00232360092038BDD98882889142F7D135
S315080017DC587802F0D3FB10F0010FF1D12B68236077
S315080017EC002038BDF8B5C3780BB90020F8BD0446FF
S315080017FCC66A00F13007012332463946407802F0B2
S3150800180C0BFCA8B90023E370236AF31AA269934266
S3150800181C10D2A57808E0A3691E440123324639463E
S3150800182C607802F0F9FB013D012DF4D80020F8BDD3
S3150800183C0120F8BD0020F8BD70B5C36A8B4214D0E0
S3150800184C04460D46FFF7CEFF064608B1304670BD76
S3150800185C01232A4604F13001607802F099FB10B195
S3150800186C01264FF0FF35E562F0E70026EEE70000AB
S3150800187C10B504460023C3704FF0FF33C362FFF75D
S3150800188CDBFF08B1042010BD04F22E20FFF70EFE74
S3150800189C4AF65523984201D0032010BD04F1660080
S315080018ACFFF709FE20F07F40084B98420CD004F154
S315080018BC8200FFF700FE20F07F40044B984201D0CF
S315080018CC022010BD002010BD002010BD464154005A
S315080018DC2DE9F04784B00E46174600230B60FFF738
S315080018EC3EFF051EC0F23581A84B53F82540002C47
S315080018FC00F03381346007F0FE0723787BB16078FB
S3150800190C02F03CFB10F0010F09D1002F00F02781E3
S3150800191C10F0040F01D00A201CE100201AE1002364
S3150800192C2370E8B2607002F083FA10F0010F01D050
S3150800193C03200FE127B110F0040F01D00A2009E1AA
S3150800194C00212046FFF794FF02281DD00026042804
S3150800195C00F0078101282DD90D20FBE0002004ABEF
S3150800196C03EB850343F8100C0135032D0ED804F14F
S3150800197C30002B0103F5DF7318440379002BEDD0E7
S3150800198C0830FFF798FDEAE70025EEE7002508E0A2
S3150800199C31462046FFF76CFF0128D8D90135032DAF
S315080019ACD5D804AB03EB850353F8106C002EEFD196
S315080019BC0320F1E704F13B00FFF778FDB0F5007F53
S315080019CC01D00D20C6E004F14600FFF76FFD8046F6
S315080019DC20B904F15400FFF76EFD8046C4F8188050
S315080019EC94F8409084F8029009F1FF33DBB2012B8E
S315080019FC01D90D20AEE009FB08F994F83D70678112
S31508001A0C002F00F0B0807B1E1F4201D00D20A1E0F4
S31508001A1C04F14100FFF74AFD8246208110F00F0FB2
S31508001A2C40F0A38004F14300FFF740FD054620B9BA
S31508001A3C04F15000FFF73FFD054604F13E00FFF7A1
S31508001A4C35FD0246002800F0928009EB000303EBF3
S31508001A5C1A139D42C0F08D80ED1AB5FBF7F5002DD3
S31508001A6C00F0898040F6F5718D4260D801274FF653
S31508001A7CF5718D4200D9032702356561E66132445A
S31508001A8C22623344A362032F53D104F15A00FFF7A1
S31508001A9C0DFD002871D1BAF1000F70D104F15C006C
S31508001AACFFF709FD6062AD0005F2FF15B8EB552F7F
S31508001ABC69D34FF0FF332361E36080232371032F2F
S31508001ACC2CD104F16000FFF7F1FC012826D1711C1A
S31508001ADC2046FFF7B1FE08BB0023237104F22E2023
S31508001AECFFF7E4FC4AF65523984217D104F1300067
S31508001AFCFFF7E1FC264B984210D104F50570FFF769
S31508001B0CDAFC244B984209D104F50670FFF7D3FC8E
S31508001B1C206104F50770FFF7CEFCE06027701E4ABB
S31508001B2C138801339BB21380E380002012E002274E
S31508001B3C9DE7BAF1000F24D04A446262022F01D104
S31508001B4C6D00B1E705EB450305F0010505EB5305FB
S31508001B5CAAE70B2004B0BDE8F0870C20FAE70020B2
S31508001B6CF8E70120F6E70D20F4E70D20F2E70D2043
S31508001B7CF0E70D20EEE70D20ECE70D20EAE70D2047
S31508001B8CE8E70D20E6E70D20E4E700BFB40C0020DB
S31508001B9C5252614172724161B80C0020F8B5066860
S31508001BAC01295DD9736999425CD20C463378022BAC
S31508001BBC30D0032B40D0012B01D00120F8BD01EB0E
S31508001BCC5105316A01EB55213046FFF735FE10B148
S31508001BDC4FF0FF30F8BD6F1CC5F30805354495F872
S31508001BEC3050316A01EB57213046FFF725FE10B10C
S31508001BFC4FF0FF30F8BDC7F308073E4496F830009F
S31508001C0C45EA002014F0010F01D00009F8BDC0F315
S31508001C1C0B00F8BD316A01EB14213046FFF70CFEB8
S31508001C2C10B14FF0FF30F8BD600000F4FF70303093
S31508001C3C3044FFF73BFCF8BD316A01EBD411304652
S31508001C4CFFF7FAFD10B14FF0FF30F8BDA00000F415
S31508001C5CFE7030303044FFF72EFC20F07040F8BD93
S31508001C6C0120F8BD0120F8BD2DE9F0410768B1F552
S31508001C7C001F02D30220BDE8F08106460C4611F07F
S31508001C8C1F0F02D00220BDE8F081316185681DB9AD
S31508001C9C3B78022B00D97D6A75B93B89B3EB541F87
S31508001CAC02D80220BDE8F0817B6AB3617561B3691D
S31508001CBC0BBB0220BDE8F081B7F80A804FEA48282A
S31508001CCC01E0A4EB080444450FD329463046FFF738
S31508001CDC65FF0546B0F1FF3F18D0012819D97B6975
S31508001CEC9842EED30220BDE8F08129463846FFF724
S31508001CFC20FCB061DAE703EB5423B3613037C4F345
S31508001D0C08043C44F4610020BDE8F0810120BDE8DC
S31508001D1CF0810220BDE8F0812DE9F84301297ED92E
S31508001D2C4369994201D302267AE017460C460546C2
S31508001D3C0378022B47D0032B57D0012B01D0022650
S31508001D4C6EE001EB5108016A01EB5821FFF774FDAF
S31508001D5C0646002864D108F10109C8F3080814F0EE
S31508001D6C010423D005EB080393F9303003F00F0375
S31508001D7C3A0102F47F621343DBB2A84488F8303088
S31508001D8C0123EB70296A01EB59212846FFF754FD0C
S31508001D9C0646002844D1C9F308094CB1C7F3071203
S31508001DACA94489F830200123EB7039E0FBB2E4E74B
S31508001DBC05EB090393F9302022F00F02C7F303272A
S31508001DCC3A43D2B2ECE7016A01EB1421FFF734FD72
S31508001DDC064628BB600000F4FF703030B9B22844C0
S31508001DECFFF774FB0123EB701AE0016A01EBD411BF
S31508001DFCFFF722FD064698B927F07047A40004F4AD
S31508001E0CFE7430342C442046FFF755FB00F0704125
S31508001E1C39432046FFF75EFB0123EB7000E00226F0
S31508001E2C3046BDE8F8832DE9F04107460668884632
S31508001E3C31B9F5688DB173699D420FD301250DE053
S31508001E4CFFF7ACFE0346012847D9B0F1FF3F49D04E
S31508001E5C7269904246D3454600E001252C460CE0B3
S31508001E6C21463846FFF79AFE034670B1012839D049
S31508001E7CB0F1FF3F36D0AC4233D0013473699C4283
S31508001E8CEED3012D2BD90224EAE74FF0FF32214677
S31508001E9C3046FFF741FF034610B9B8F1000F0ED1D3
S31508001EACA3B9F46033697269023A934201D2013BD1
S31508001EBC3361337943F001033371234612E022462A
S31508001ECC41463046FFF728FF0346E9E7012B01D0C8
S31508001EDC012307E04FF0FF3304E0012302E000235F
S31508001EEC00E000231846BDE8F081F8B50E460468F4
S31508001EFC012930D90746114663699E4201D302224D
S31508001F0C2AE05AB14FF0FF322046FFF705FF02468A
S31508001F1C20B121E063692E469D421DD231463846D2
S31508001F2CFFF73CFE0546C8B1012819D0B0F1FF3FB2
S31508001F3C18D0002231462046FFF7EEFE024658B965
S31508001F4C2369B3F1FF3FE5D001332361237943F0CD
S31508001F5C01032371DEE702221046F8BD0022FBE7D7
S31508001F6C0222F9E70122F7E72DE9F8430668036927
S31508001F7C03F12005836913B90420BDE8F883B5F588
S31508001F8C001F02D30420BDE8F88388460446C5F32F
S31508001F9C08078FB901338361416941B93389B3EBBA
S31508001FAC551F09D8002383610420BDE8F88373897B
S31508001FBC013B13EA552307D0256107F1300846443F
S31508001FCCE6610020BDE8F883FFF7E8FD81460128A5
S31508001FDC48D9B0F1FF3F48D0736998423AD3B8F163
S31508001FEC000F04D10023A3610420BDE8F8836169BE
S31508001FFC2046FFF718FF814610B90720BDE8F8837D
S3150800200C012835D0B0F1FF3F35D03046FFF7EAFB53
S3150800201CA0BB4FF40072002106F13000FFF76DFAF1
S3150800202C49463046FFF785FAF0624FF00008738987
S3150800203C98450BD20123F3703046FFF7D3FB00BB50
S3150800204C08F10108F36A0133F362F0E7F36AA3EBCC
S3150800205C0803F362C4F8149049463046FFF769FA48
S3150800206CA061A9E70220BDE8F8830120BDE8F88342
S3150800207C0220BDE8F8830120BDE8F8830120BDE8FD
S3150800208CF8830120BDE8F883F8B504460F460668C0
S3150800209C0021FFF7E9FD0246C0B9002508E0013525
S315080020ACBD4213D001212046FFF75EFF024668B9F0
S315080020BCA1693046FFF7C0FB024638B9E3691B78BD
S315080020CCE52BECD0002BEAD00025EBE7042A01D04F
S315080020DC1046F8BD0722FBE72DE9F8430446884667
S315080020EC07684FF0FF094E4604252EE00F2B19D131
S315080020FC12F0400F06D091F80D9002F0BF0223693A
S3150800210C63621646B24201D0FF2618E04B7B99450E
S3150800211C01D0FF2613E0A06AFFF73EFA88B3013E0A
S3150800212CF6B20CE026B90846FFF70BFB81452BD017
S3150800213C4FF0FF33636227E0FF2600E0FF260021FD
S3150800214C2046FFF711FF0546F0B9A169E1B13846FB
S3150800215CFFF772FB0546B8B9E1690A789AB1CB7AEA
S3150800216C03F03F03A371E52AE6D02E2AE6D023F026
S3150800217C2000082814BF002001204045B6D0FF26B1
S3150800218CDDE7FF26DBE704250DB10023A36128460E
S3150800219CBDE8F88370B5044605680669416AB1F16D
S315080021ACFF3F1CD0FFF760FD0346B3B9A16928466B
S315080021BCFFF742FB034670B9E269E521117001226B
S315080021CCEA702269964206D900212046FFF7CCFE12
S315080021DC03460028EAD0042B03D0184670BD00230A
S315080021ECE3E70223F9E700002DE9F04F83B0064632
S315080021FC8A46D1F80090856A002412E0013709EB6B
S3150800220C070219F807302F2BF8D05C2BF6D0CAF832
S3150800221C00201F2822D84FF0040823E025F8148044
S3150800222C3C46671C19F804001F28E8D92F28E6D065
S3150800223C5C28E4D0FE2C00F2DD80012100F0E2FFE0
S3150800224C8046002800F0D8807F28E7D801466B48DE
S3150800225CFFF767F90028E1D0062012E04FF00008D6
S3150800226C00E0013C44B104F10043013B35F813305E
S3150800227C202BF6D02E2BF4D0002325F814301CB9BD
S3150800228C062003B0BDE8F08F0B222021306AFFF739
S3150800229C34F9002300E0013335F81320202AFAD04C
S315080022AC2E2AF8D01BB148F0030800E0013C6CB1AB
S315080022BC04F10042013A35F812202E2AF6D14FF0D5
S315080022CC080B4FF0000ACDF804A00AE0A2464FF01E
S315080022DC080B0022019204E04C450BD048F0030889
S315080022EC4B4603F1010935F8137057B3202FF5D077
S315080022FC2E2FF1D0DA450FD24C450DD07F2F3FD873
S3150800230C002F4AD148F003085F27336A03F80A708E
S3150800231C4B460AF1010AE4E7BBF10B0F0FD04C450B
S3150800232C01D048F003084C450BD3019B9B00DBB24C
S3150800233C019323464FF00B0B4FF0080AD1E748F0F0
S3150800234C0308336A1A78E52A43D0BBF1080F43D041
S3150800235C019901F00C020C2A43D001F00303032B5C
S3150800236C3FD018F0020F06D1019B03F00303012B93
S3150800237C3AD0042A3BD0336A83F80B80002080E7D6
S3150800238C0021384600F03EFF074618B1A0F1800739
S3150800239C1B4BDF5D48F00208B2E739461948FFF7D0
S315080023ACC0F80028AED1A7F141039BB2192B04D86B
S315080023BC019B43F002030193A7E7A7F161039BB2C4
S315080023CC192BA2D8019B43F001030193203FBFB2FE
S315080023DC9BE705221A70B8E7019B9B00DBB20193B9
S315080023ECB6E748F00208BCE748F01008C1E748F021
S315080023FC0808C0E7062044E7062042E754490008C7
S3150800240CC448000860490008F8B500238B75836931
S3150800241C002B6BD00D460646436AB3F1FF3F13D02B
S3150800242C836A00249F1C188858B1002100F0EAFE24
S3150800243C30B1FE2C0CD82A1990753B460134F1E7BD
S3150800244C00242C440023A375AC7D0022134612E00D
S3150800245C0024F6E7E52317E014B9A8182E27877584
S3150800246CA8182E274772013210E010271CE0A8186E
S3150800247C837501320B460A2B1BD8F069591CC35CB1
S3150800248C202BF7D0052BE5D00929E5D0A8184372DF
S3150800249C002CEED1A3F14100C0B21928E7D8F06997
S315080024AC007B0829E1D808270742E0D02033DBB2A5
S315080024BCDDE734B9AB1800219975F3691B7B03B9B1
S315080024CC0A462A4400235372F369DB7A2B72F069A5
S315080024DC1C30FEF7F0FF2860F0691830FEF7E6FFAF
S315080024ECA880F0691630FEF7E1FFE880F8BD000019
S315080024FC2DE9F0478146884601F11A00FEF7D6FF0A
S3150800250CB0BB98F8005005F03F05013D05EB4503B7
S3150800251C05EB83050127002404E04FF6FF73984268
S3150800252C2FD101340C2C17D81C4B185D4044FEF7E0
S3150800253CBDFF0646002FF0D0FE2D1CD800F07EFEFF
S3150800254C074605F1010A39F8150000F077FE8742AF
S3150800255C14D137465546E4E798F8003013F0400F87
S3150800256C12D0A7B139F81530A3B90120BDE8F08708
S3150800257C0020BDE8F0870020BDE8F0870020BDE804
S3150800258CF0870020BDE8F0870120BDE8F087012020
S3150800259CBDE8F0870020BDE8F08700BF4449000875
S315080025AC2DE9F8430446D0F800800021FFF75CFBC0
S315080025BC064600285ED14FF0FF3363624FF0FF09E1
S315080025CC4F460AE04FF0FF336362FF27002120468F
S315080025DCFFF7CAFC064600284CD1A1694046FFF70E
S315080025EC2BF90646002845D1E5692B78002B40D0F7
S315080025FCE97A01F03F02A271E52BE3D011F0080F3E
S3150800260C01D00F2ADED10F2A14D027B92846FFF796
S3150800261C98F881452ED0216ACB7A13F0010F04D194
S3150800262C0B222846FEF76EFF20B34FF0FF3363628A
S3150800263CFF27CBE7A06A0028C8D013F0400F06D0B6
S3150800264C95F80D9003F0BF03226962621F46BB42E0
S3150800265C01D0FF27BAE76B7B994501D0FF27B5E771
S3150800266C2946FFF745FF10B1013FFFB2AEE7FF273A
S3150800267CACE704263046BDE8F88330B583B004468B
S3150800268C0191056801E001330193019B1A782F2A01
S3150800269CF9D05C2AF7D00022A2601B781F2B1DD913
S315080026AC01A92046FFF7A0FD0346F8B92046FFF717
S315080026BC77FF236ADA7A0346D8B912F0040F15D1D4
S315080026CCA37913F0100F1BD02169C1F3080130311F
S315080026DC29442846FEF739FFA060E1E7236A8022E1
S315080026ECDA7200212046FFF7BFFA0346184603B0F4
S315080026FC30BD0428FAD112F0040FF7D10523F5E7FB
S3150800270C0523F3E72DE9F04784B00668D0F820A036
S3150800271CD0F828809AF80B3013F0A00F05D04FF09C
S3150800272C0609484604B0BDE8F087002400E00134E9
S3150800273C38F81430002BFAD105460C22514601A85C
S3150800274CFEF7D2FE9DF80F3013F0010F1ED00023B2
S3150800275C8AF80B30AB620127632F0CD83B464246EE
S3150800276C01A95046FEF79AFF2846FFF719FF81463E
S3150800277C08B90137F0E7642F60D0B9F1040FD0D14E
S3150800278C9DF80F308AF80B30C5F828809DF80F3065
S3150800279C13F0020F2AD00C342A4BA3FB0434A408DA
S315080027AC013421462846FFF76FFC814608B9013CDF
S315080027BC1ED1B9F1000FB4D1A9693046FFF73CF820
S315080027CC81460028ADD120220021E869FEF795FE46
S315080027DC0B22296AE869FEF787FEEA692B6ADB7A17
S315080027EC03F0180313730123F3709AE70124D8E74F
S315080027FC2969A1EB44112846FFF736FA81460028C9
S3150800280CD7D1286AFEF79DFF0746A9693046FFF718
S3150800281C13F881460028CCD13B46E2B2E969A86A8E
S3150800282CFEF700FF0123F37000212846FFF79CFBF7
S3150800283C81460028BDD1013CE7D1BAE74FF007091C
S3150800284C6FE700BF4FECC44E70B50446FEF7CAFFDF
S3150800285C054648B92378032B08D000221146607820
S3150800286C01F030FC00B10125284670BD2379012BF7
S3150800287CF3D104F130064FF4007200213046FEF70E
S3150800288C3CFE4AF6552104F22E20FEF71FFE0F4990
S3150800289C3046FEF71FFE0E4904F50570FEF71AFEC4
S315080028AC216904F50670FEF715FEE16804F5077054
S315080028BCFEF710FEE2690132E262012331466078C6
S315080028CC01F0AAFB00232371C7E700BF52526141EE
S315080028DC7272416110B584B001900091144604A837
S315080028EC40F8041DFEF73BFF002818DB0E4B53F887
S315080028FC20300BB100221A70019B0BB100221A7002
S3150800290C019B094A42F8203063B1012C01D0002002
S3150800291C06E0002201A96846FEF7DAFF00E00B2064
S3150800292C04B010BD0020FBE7B40C00202DE9F043E1
S3150800293C93B00191002800F0AE8004461646002399
S3150800294C036002F01F073A4606A901A8FEF7C0FF66
S3150800295C0546002840F0A080069B079303AB0F930F
S3150800296C4F4B1193019907A8FFF787FE054620B927
S3150800297C0F9B93F90B30002B2FDB16F01C0F79D01D
S3150800298C002D31D0042D2AD047F0080715B917F0B9
S3150800299C080F35D14DB917F0080F01D047F02007AD
S315080029AC069BDB6A23620E9B6362002D74D1069E1E
S315080029BCDDF8388041463046FEF7C7FDA06008F1C1
S315080029CC1C00FEF778FDE060002363746361E36125
S315080029DC27742660F388A3805EE00625CDE707A852
S315080029ECFFF790FE0546CFE79DF8223013F0110F3E
S315080029FC04D116F0040FC9D00825C7E70725C5E783
S31508002A0C284E31460E980E30FEF764FD31460E9868
S31508002A1C1630FEF75FFD20220E9BDA72069EDDF855
S31508002A2C388041463046FEF790FD814600224146E5
S31508002A3C3046FEF79DFD00210E981C30FEF74AFD28
S31508002A4C0122069BDA70B9F1000FA3D0069BDE6A49
S31508002A5C0022494607A8FFF748FA0546002899D1E7
S31508002A6C31460698FEF7E8FE054609F1FF33069A45
S31508002A7CD3608FE7002D8DD19DF8223013F0100FFF
S31508002A8C07D116F0020F85D013F0010F82D0072557
S31508002A9C80E704257EE70925284613B0BDE8F083B0
S31508002AACBC0C0020000061482DE9F04F85B00446A7
S31508002ABC8846164699460023C9F8003003A9FEF73E
S31508002ACC77FE074630B9677C27B9237C13F0010FCC
S31508002ADC04D10727384605B0BDE8F08FE36862696C
S31508002AEC9B1AB34253D21E4651E0A1692046FFF702
S31508002AFC55F85EE002276774ECE701276774E9E787
S31508002B0C02276774E6E701276774E3E74FF4007258
S31508002B1C04F1280108EB4020FEF7E6FC74E0E269B4
S31508002B2C019B934219D0237C13F0400F0BD0012341
S31508002B3C04F12801687801F06FFA002867D1237C24
S31508002B4C23F0400323740123019A04F12801039806
S31508002B5C407801F01DFA00285CD1019BE36161699C
S31508002B6CC1F30801C1F50075AE4200D235462831CD
S31508002B7C2A4621444046FEF7B7FCA84463692B4411
S31508002B8C6361D9F800302B44C9F80030761B002E47
S31508002B9CA0D06369C3F30802002AE0D1039AB2F8FD
S31508002BAC0AA00AF1FF3A1AEA532A08D1002B9CD13B
S31508002BBCA06801289ED9B0F1FF3F9ED0A061039D65
S31508002BCCA1692846FEF7B5FC002899D00AEB000344
S31508002BDC01935FEA562BA2D00AEB0B036A89934240
S31508002BEC01D9A2EB0A0B5B46019A4146687801F0BB
S31508002BFCCFF9002887D1237C13F0400F04D0E06965
S31508002C0C019BC01A834581D84FEA4B25B5E70127A6
S31508002C1C67745FE7012767745CE72DE9F04F85B0A9
S31508002C2C04468846164699460023C9F8003003A977
S31508002C3CFEF7BEFD074630B9677C27B9237C13F02F
S31508002C4C020F04D10727384605B0BDE8F08F636933
S31508002C5CF3425FD3DE435DE000212046FFF7E3F83D
S31508002C6C6CE0A1692046FFF7DEF867E00227677477
S31508002C7CE9E701276774E6E70123E26904F128010D
S31508002C8C0398407801F0C8F920B9237C23F0400357
S31508002C9C237462E001276774D5E702276774D2E7C5
S31508002CAC01276774CFE74FF4007208EB412104F152
S31508002CBC2800FEF719FC237C23F0400323746EE0EE
S31508002CCCE3699B4503D06269E3689A4269D3C4F801
S31508002CDC1CB06069C0F30800C0F50075AE4200D29E
S31508002CEC354628302A4641462044FEF7FDFB237C10
S31508002CFC43F040032374A84463692B446361E26878
S31508002D0C934238BF1346E360D9F800302B44C9F810
S31508002D1C0030761B002E51D06369C3F30802002AD3
S31508002D2CD7D1039AB2F80AA00AF1FF3A1AEA532A3B
S31508002D3C0FD1002B95D1A06800288DD000283DD046
S31508002D4C012893D0B0F1FF3F93D0A061A36803B9D3
S31508002D5CA060237C13F0400F8ED1039B0193A169CD
S31508002D6C1846FEF7E6FB8346002896D0D344750A28
S31508002D7CA6D00AEB0503019A5289934201D9A2EB14
S31508002D8C0A052B465A4641460198407801F044F903
S31508002D9C002885D1E169A1EB0B018D4283D86D0220
S31508002DACA9E701235A4604F128010198407801F055
S31508002DBCEFF800288BD00127677444E7237C43F08F
S31508002DCC200323743FE770B582B004460E460A29E1
S31508002DDC0DD06368002B08DB5D1C23441E733C2D49
S31508002DEC09DC6560A3680133A36002B070BD0D21D0
S31508002DFCFFF7E9FFEDE701AB2A4604F10C01206861
S31508002E0CFFF70BFF019B9D4202D04FF0FF35E8E719
S31508002E1C0025E6E730B583B0044601A9FEF7C8FCE1
S31508002E2C0346C8B9227C12F0200F15D012F0400FB9
S31508002E3C0CD00123E26904F128010198407801F0CD
S31508002E4CEBF888BB237C23F040032374216A019892
S31508002E5CFEF7F2FC034610B1184603B030BD656A9E
S31508002E6CEB7A43F02003EB72A26829462068FEF73A
S31508002E7C7FFBE16805F11C00FEF72CFB0B4905F1FD
S31508002E8C1600FEF727FB002105F11200FEF71EFBC4
S31508002E9C0122019BDA700198FFF7D6FC0346227CC7
S31508002EAC22F020022274D7E70123D5E700006148F7
S31508002EBC10B582B00446FFF7ADFF034610B11846AD
S31508002ECC02B010BD01A92046FEF772FC0346002885
S31508002EDCF5D100222260F2E72DE9F04182B00446D2
S31508002EEC0E4601A9FEF764FC0746002840F0A280AE
S31508002EFC677C002F40F09E80E368B34204D2227CA4
S31508002F0C12F0020F00D11E46636900226261002E80
S31508002F1C65D0019AB2F80A804FEA482873B1721E36
S31508002F2CB2FBF8F2013BB3FBF8F18A4206D3C8F1BF
S31508002F3C000213406361F61AA56902E0A56815B18B
S31508002F4CA56135BB4CE000212046FEF76CFF054613
S31508002F5C012804D0B0F1FF3F04D0A060F0E70227A7
S31508002F6C677467E00127677464E029462046FEF714
S31508002F7C15FE0546B5F1FF3F28D0012D29D9019B31
S31508002F8C5B699D4225D2A561636943446361A6EBDF
S31508002F9C080646450BD9237C13F0020FE5D02946C3
S31508002FAC2046FEF740FF05460028E3D146466369EE
S31508002FBC33446361C6F30803002B3FD029460198B6
S31508002FCCFEF7B7FA40B90227677433E0012767742E
S31508002FDC30E0022767742DE000EB562500E000254B
S31508002FEC6369C3F30803E3B1E269954219D0237CFC
S31508002FFC13F0400F0BD0012304F1280101984078F7
S3150800300C01F00AF8E0B9237C23F04003237401236A
S3150800301C2A4604F128010198407800F0B9FF90B9C6
S3150800302CE5616369E268934204D9E360237C43F063
S3150800303C20032374384602B0BDE8F0810025CFE79B
S3150800304C01276774F6E701276774F3E730B591B083
S3150800305C01900D46002205A901A8FEF739FC044685
S3150800306C10B1204611B030BD02AB0D930B4B0F932C
S3150800307C019905A8FFF701FB04460028F1D10D9B21
S3150800308C93F90B30002B06DB002DEAD0294605A850
S3150800309CFFF7BAF9E5E70624E3E700BFBC0C002006
S315080030AC70B59CB00190022205A901A8FEF710FC88
S315080030BC059B1193044610B120461CB070BD02AB9B
S315080030CC1993264B1B93019911A8FFF7D6FA0446B8
S315080030DC0028F1D1199B93F90B30002B23DB9DF8B3
S315080030EC4A3013F0010F20D10CBB059E18993046B7
S315080030FCFEF72BFA05469DF84A3013F0100F17D039
S3150800310C06960890002106A8FEF7AEFD044678B987
S3150800311C002106A8FEF7E0FF034600B90723042B97
S3150800312C06D01C4604E00624DEE70724DCE7002567
S3150800313C002CC1D111A8FFF72DF8044600B935B9F2
S3150800314C002CB9D10598FFF77FFB0446B4E700229B
S3150800315C294611A8FEF7C9FE0446F1E7BC0C002067
S3150800316C2DE9F04182B080460E46174605460024E6
S3150800317C731E9C4214DA6B46012201A93846FFF7E6
S3150800318C93FC009B012B0BD19DF804300D2BEFD033
S3150800319C6A1C2B7001340A2B01D01546E8E7154634
S315080031AC00232B701CB1404602B0BDE8F08100200C
S315080031BCFAE710B594B004460191002302930393E1
S315080031CC03E0013401A8FFF7FEFD21780029F8D1A8
S315080031DC029A002A0CDB6B4604A90198FFF71DFD21
S315080031EC48B9009B029A9A4208D1039814B010BDAC
S315080031FC4FF0FF30FAE74FF0FF30F7E74FF0FF30AC
S3150800320CF4E700007F2816D931B1FF2812D8803888
S3150800321C094B33F81000704700237F2B07D8064A52
S3150800322C32F81320904202D001339BB2F5E7803373
S3150800323CD8B270470020704768490008B0F5805F1F
S3150800324C06D2224B1A881AB3904221D3F0B406E060
S3150800325C1F4BF7E72B461A88CAB1904217D31D1D88
S3150800326C5B88190ADBB29C18A04204DB0029F1D151
S3150800327C05EB4303EFE7082909D8DFE801F0050A4F
S3150800328C101316191C1F2200861A35F81600F0BCE6
S3150800329C7047821A02F00103C01A80B2F7E7103899
S315080032AC80B2F4E7203880B2F1E7303880B2EEE726
S315080032BC1A3880B2EBE7083080B2E8E7503880B2AB
S315080032CCE5E7A0F5E35080B2E1E700BF684A0008DD
S315080032DC5C4C00080022014B5A707047BC0E00204B
S315080032EC034BFE22DA7018710222A3F844207047A9
S315080032FCBC0E002010B5054C00232370FFF7EAFF1F
S3150800330CFF23E3700123A4F8443010BDBC0E002043
S3150800331C064BFF22DA7000221A71597859719A7184
S3150800332CDA711A720622A3F844207047BC0E0020E4
S3150800333C08B50020FFF7D4FF08BD0000074BFF2295
S3150800334CDA70074A9A6400221A715A719A7107221E
S3150800335CC3F807200822A3F844207047BC0E0020A7
S3150800336C184D0008044BFF22DA7042689A64012251
S3150800337CA3F84420704700BFBC0E002008B53120C6
S3150800338CFFF7AEFF08BD000038B5084CFF23E37005
S3150800339C002525716571FDF7A7FCA071E5712572ED
S315080033AC65720723A4F8443038BD00BFBC0E002054
S315080033BC38B5FDF74DFDE8B1FFF78CFF0F4C01252D
S315080033CC2570FF23E3701023237100236371FDF727
S315080033DC8BFCA071FDF79AFCE071FDF797FCC0F326
S315080033EC072020726572A5720823A4F84430FDF7ED
S315080033FCC1FA38BD1020FFF773FF38BDBC0E00208C
S3150800340C38B505464478FDF76FFC0138844210DC64
S3150800341C0A4C6A78A16C201DFDF720F8FF23E3708F
S3150800342C6A78A36C1344A3646B780133A4F844300C
S3150800343C38BD2220FFF754FF38BD00BFBC0E002054
S3150800344C38B504464578FDF74FFC0138854211DC42
S3150800345C61680A4DA9646278281DFCF7FFFFFF23F3
S3150800346CEB706278AB6C1344AB6463780133A5F8E4
S3150800347C443038BD2220FFF733FF38BDBC0E002080
S3150800348CF8B505461746002406E015F8013B1C441A
S3150800349CE4B2FDF752FC31464E1E0029F5D13C60CC
S315080034AC0120F8BD10B5084CFF23E370E21D4168F6
S315080034BCA06CFFF7E5FF207100236371A371082345
S315080034CCA4F8443010BD00BFBC0E002038B5054624
S315080034DC0D4B9C6CFDF708FC6A1C411E2046FDF73B
S315080034EC4DFA60B1084CFF23E370FDF7FDFB01387C
S315080034FCA36C0344A3640123A4F8443038BD3120DB
S3150800350CFFF7EEFE38BD00BFBC0E002038B50446EA
S3150800351C4578FDF7E9FB023885420EDC114BFF2294
S3150800352CDA700122A3F84420617851B9FDF736FA0E
S3150800353C90B93120FFF7D4FE38BD2220FFF7D0FE14
S3150800354C38BDA21C074B986CFDF718FA28B16178A0
S3150800355C044A936C0B44936438BD3120FFF7C0FEC4
S3150800356C38BD00BFBC0E002008B54168074B986CE7
S3150800357CFDF708FA30B1054BFF22DA700122A3F8E1
S3150800358C442008BD3120FFF7ABFE08BDBC0E002059
S3150800359C08B5FCF749FF034BFF22DA700122A3F8A2
S315080035AC442008BDBC0E002008B589B2FDF784FB83
S315080035BC08BD0000054B00221A709A6483F8432054
S315080035CCA3F844209A705A70704700BFBC0E0020AE
S315080035DC034B1B780BB1012070470020704700BFC6
S315080035ECBC0E00200022024B83F84320704700BF14
S315080035FCBC0E002008B50378FF2B04D0354A127888
S3150800360C012A14D008BDFFF7D3FE324B93F843308A
S3150800361C012B5AD02F4BB3F944100029F2DD18466A
S3150800362C012380F843300330FFF7BEFFEAE7C93BB6
S3150800363C352B46D8DFE803F03345454245453F363A
S3150800364C3C39454545454545454545454545454525
S3150800365C4545454545454545454545454545454500
S3150800366C4545241E1B2145454527452A2D30FFF780
S3150800367CC7FECAE7FFF7E4FEC7E7FFF773FEC4E722
S3150800368CFFF710FFC1E7FFF759FEBEE7FFF750FE3D
S3150800369CBBE7FFF73DFEB8E7FFF72CFEB5E7FFF7EC
S315080036AC15FFB2E7FFF732FFAFE7FFF76DFEACE7A2
S315080036BCFFF75AFFA9E7FFF76BFFA6E7FFF75EFED2
S315080036CCA3E72020FFF70CFE9FE71020FFF708FE64
S315080036DCA0E700BFBC0E002000B5C7B04FF48C7233
S315080036EC0021684600F058FF69460948FFF7AEFC0A
S315080036FC40B9009B53B19DF8083013F0100F02D156
S3150800370C012000E0002047B05DF804FB0020FAE732
S3150800371C304D000800487047304D000808B507487A
S3150800372C002380F828320A220549FFF7FFF818B952
S3150800373C0122024B83F8282208BD00BF080F00207F
S3150800374C204D000810B50D4B93F82832012B10D0DC
S3150800375CFDF758F900F164044021094800F098F97E
S3150800376C18B9FDF74FF98442F6D20648FFF798FCCC
S3150800377C10BD0248FFF79CFBEAE700BF080F0020C4
S3150800378C00440040304D000808B5054B93F8283224
S3150800379C012B00D008BD0248FFF78AFBFAE700BFE9
S315080037AC080F002010B504460F4B93F82832012B4E
S315080037BC15D10D49FFF7FDFC002810DA0A4800233D
S315080037CC80F82832FFF774FB09E0084800F05CF92A
S315080037DC8021064800F05CF90028F9D001342178DC
S315080037EC0029F2D110BD00BF080F0020004400408C
S315080037FC82B00023019300932C4A136843F4803358
S3150800380C13602A4B1B6803F400330093019B0133A6
S3150800381C0193009B1BB9019BB3F5A06FF1D1234B08
S3150800382C1B6813F4003F06D001230093009B012B61
S3150800383C04D002B0704700230093F7E71C4B1A68B4
S3150800384C42F010021A601A6822F003021A601A680B
S3150800385C42F002021A60A3F580535A685A605A68F5
S3150800386C5A605A6842F480625A605A6822F47C128A
S3150800387C5A605A6842F4E8125A601A6842F0807222
S3150800388C1A600A4B1B6813F0007FFAD0074B5A686C
S3150800389C22F003025A605A6842F002025A60034B3D
S315080038AC5B6803F00C03082BF9D1C2E70010024041
S315080038BC0020024008B5FFF79BFF08BD08B5104B62
S315080038CC1A6842F001021A6059680E4A0A405A6090
S315080038DC1A6822F0847222F480321A601A6822F46A
S315080038EC80221A605A6822F4FE025A604FF41F02AC
S315080038FC9A60FFF7DFFF4FF00062034B9A6008BD32
S3150800390C001002400000FFF800ED00E0F0B4CB78A0
S3150800391C03F00F02154613F0100F01D08D781543DE
S3150800392C0B78E3B10668002301E042610133072BEB
S3150800393C14D801229A400C8832EA0404F6D19C0069
S3150800394C0F27A74026EA070605FA04F42643CC787F
S3150800395C282CEAD0482CE9D10261E7E706600B88E7
S3150800396CFF2B20D94668002302E0426115E001339B
S3150800397C072B17D803F108040122A2400C8832EA57
S3150800398C0404F4D19C000F27A74026EA070605FA7B
S3150800399C04F42643CC78282CE7D0CC78482CE6D1EE
S315080039AC0261E4E74660F0BC70470161704741610B
S315080039BC7047000029B9054A936923EA000090610B
S315080039CC7047024A93691843906170470010024089
S315080039DC29B9054AD36923EA0000D0617047024A1F
S315080039ECD3691843D0617047001002402DE9F041A5
S315080039FC038803F44153B1F800C0B1F80280B1F85A
S31508003A0C04E0CF880E894D898C89CA894CEA080C42
S31508003A1C4EEA0C0E47EA0E073E4335432C43224327
S31508003A2C13430380838B9BB223F400639BB283837B
S31508003A3C0B8A0382BDE8F08131B903889BB223F067
S31508003A4C40039BB20380704703889BB243F0400344
S31508003A5C0380704781817047808980B2704731B97D
S31508003A6C03889BB223F400539BB2038070470388E8
S31508003A7C9BB243F40053038070470389194201D162
S31508003A8C0020704701207047C1F3080181807047F8
S31508003A9C0388194201D100207047012070470000A5
S31508003AAC024A137843F00103137070470100002093
S31508003ABC30B587B0154D00212846FFF7BDFF002409
S31508003ACCADF804404FF48273ADF80630ADF80840F3
S31508003ADCADF80A40ADF80C404FF40073ADF80E3053
S31508003AEC0823ADF81030ADF812400723ADF81430A2
S31508003AFC01A92846FFF77AFF21462846FFF7AFFFAC
S31508003B0C01212846FFF798FF07B030BD0038004062
S31508003B1C30B583B01E4C4FF480512046FFF745FF55
S31508003B2C4FF40045ADF8045003238DF806301023E6
S31508003B3C8DF8073001A92046FFF7E8FE29462046EE
S31508003B4CFFF733FF002410E002211248FFF795FF18
S31508003B5C0028F9D0FF210F48FFF77CFF01210D48FB
S31508003B6CFFF78BFF0028F9D00134092CECD94FF458
S31508003B7C0043ADF8043003238DF8063018238DF86E
S31508003B8C073001A90248FFF7C1FE03B030BD00BFDC
S31508003B9C000C01400038004070B586B001210820A1
S31508003BACFFF708FF01214FF48040FFF711FF4FF490
S31508003BBC8056ADF8006010238DF8033003258DF878
S31508003BCC0250254C69462046FFF7A0FE3146204692
S31508003BDCFFF7EBFE4FF42043ADF800308DF802509A
S31508003BEC18238DF8033069462046FFF78FFE4FF4ED
S31508003BFC8043ADF8003048238DF8033069462046DB
S31508003C0CFFF784FE0024ADF804404FF48273ADF838
S31508003C1C0630ADF80840ADF80A40ADF80C404FF444
S31508003C2C0073ADF80E303823ADF81030ADF81240ED
S31508003C3C0723ADF81430094D01A92846FFF7D6FE1F
S31508003C4C21462846FFF70BFF01212846FFF7F4FE0D
S31508003C5CFFF75EFF06B070BD000C0140003800404F
S31508003C6C08B501460648FFF7F5FE01210448FFF79B
S31508003C7C04FF0028F9D00248FFF7EEFEC0B208BDD3
S31508003C8C0038004038B5FCF7BDFE00F5FA75FF2084
S31508003C9CFFF7E6FF0446FF2803D0FCF7B3FE854280
S31508003CACF5D8FF2C14BF0020012038BD08B54FF4F9
S31508003CBC80510348FFF779FEFF20FFF7D1FF08BDB7
S31508003CCC000C014010B54FF480510848FFF76FFE01
S31508003CDCFF20FFF7C5FFFFF7D5FF10B101242046DB
S31508003CEC10BD0446FFF7E2FFF9E700BF000C0140E0
S31508003CFC38B504460D4610F0800F06D1FFF7D6FFEF
S31508003D0CFFF7E0FF50B9FF2038BD00F07F04002113
S31508003D1C3720FFF7EDFF0128F6D8EFE744F040000F
S31508003D2CFFF79EFF280EFFF79BFFC5F30740FFF72B
S31508003D3C97FFC5F30720FFF793FFE8B2FFF790FF4D
S31508003D4C94B10120082C11D0FFF78AFF0C2C0FD048
S31508003D5C0A24FF20FFF784FF10F0800FD4D0631ECF
S31508003D6C13F0FF04F5D138BD9520EBE78720EBE778
S31508003D7CFF20FFF775FFEBE710B50446FF20FFF7AA
S31508003D8C6FFF207010BDF8B505460E46FCF73AFED7
S31508003D9C00F16407FF20FFF763FF0446FF2803D1F1
S31508003DACFCF730FE8742F5D8FE2C01D00020F8BD72
S31508003DBC6C1C2846FFF7E0FF20460235FFF7DCFFB0
S31508003DCC023EF5D1FF20FFF74BFFFF20FFF748FF18
S31508003DDC0120F8BD70B505460C46FFF753FF0346A0
S31508003DEC08B9184670BD2046FFF73AFFFD2C1BD0C4
S31508003DFC4FF400762C4614F8020BFFF731FF68785F
S31508003E0CFFF72EFF2546023EF4D1FF20FFF728FFC9
S31508003E1CFF20FFF725FFFF20FFF722FF00F01F000A
S31508003E2C052803D00023DCE70123DAE70123D8E7CA
S31508003E3C002840F09A80F0B583B004464C4B1B78AA
S31508003E4C13F0020F04D04A4B1878C0B203B0F0BD79
S31508003E5CFFF7A2FE4FF480514648FFF7A8FD002154
S31508003E6C0846FFF745FF0546012810D0424B1C6053
S31508003E7CFFF71CFF002C75D03D4A137803F0FE03A0
S31508003E8C1370FFF715FE3A4B1878C0B2DEE7FCF74D
S31508003E9CB9FD00F57A764FF4D5710820FFF728FF9F
S31508003EAC012846D00021A920FFF722FF012854D962
S31508003EBC2F46FCF7A7FD864205D900212846FFF7B1
S31508003ECC17FF0028F5D1FCF79DFD8642CED94FF495
S31508003EDC00711020FFF70CFF0028C7D13C46C5E738
S31508003EECFF20FFF7BDFE02AB2B4403F8040C01358B
S31508003EFCEDB2032DF4D99DF80630012BB6D19DF8F9
S31508003F0C0730AA2BB2D1FCF77DFD864206D94FF0B5
S31508003F1C8041A920FFF7ECFE0028F4D1FCF772FDCE
S31508003F2C8642A3D900213A20FFF7E2FE054658B18E
S31508003F3C9CE72546DDE7FF20FFF792FE02AB2B44F4
S31508003F4C03F8040C0135EDB2032DF4D99DF80430B1
S31508003F5C13F0400F04D00C2488E70227A925A8E7FC
S31508003F6C042483E7FFF79CFD8DE70120704700BF0B
S31508003F7C01000020000C01403411002018B9034B35
S31508003F8C1878C0B270470120704700BF01000020A6
S31508003F9C08B10420704738B50D461C460BB90420E9
S31508003FAC38BD1B4B1B7813F0010F01D0032038BD0D
S31508003FBC184B1B6813F0080F00D15202012C18D0AD
S31508003FCC11461220FFF794FE68B94FF40071284683
S31508003FDCFFF7D9FE18B105F50075013CF5D100219E
S31508003FEC0C20FFF785FEFFF761FE201C18BF012089
S31508003FFC38BD11461120FFF77BFE0028F3D14FF48C
S3150800400C00712846FFF7BFFE0028ECD00024EAE72B
S3150800401C010000203411002008B10420704770B547
S3150800402C0D4616461C460BB9042070BD234B1B784F
S3150800403C13F0010F01D0032070BD204B1B7813F031
S3150800404C040F01D0022070BD1D4B1B6813F0080F1E
S3150800405C00D15602012C1BD013F0060F26D131467F
S3150800406C1920FFF745FE68B9FC212846FFF7B2FE72
S3150800407C18B105F50075013CF6D1FD210020FFF7B6
S3150800408CA9FEC0B1FFF712FE201C18BF012070BD97
S3150800409C31461820FFF72CFE0028F3D1FE212846BE
S315080040ACFFF798FE0028EDD00024EBE72146972071
S315080040BCFFF71EFED3E70124E4E700BF010000204A
S315080040CC3411002030B585B018B10424204605B04B
S315080040DC30BD924B1B7813F0010F01D00324F5E782
S315080040EC14460E2900F20B81DFE811F00F001600BA
S315080040FC09015F0009010901090109010901090101
S3150800410CBB00C200D100DF00F100FFF7DBFD002881
S3150800411C40F0F7800124A8E000210920FFF7E8FD0C
S3150800412C08B10124A1E010216846FFF72CFE0028EF
S3150800413C00F0E9809DF800309B09012B24D09DF8EE
S3150800414C053003F00F039DF80A2003EBD2139DF8F4
S3150800415C0920520002F006021344DBB20233DBB22A
S3150800416C9DF808109DF80720920002EB91129DF815
S3150800417C0610890201F440610A440132093B02FA2D
S3150800418C03F32360002470E09DF809309DF808209D
S3150800419C03EB02239DF80720120402F47C12134445
S315080041AC01339B02236000245FE05D4B1B6813F010
S315080041BC040F21D000218D20FFF79AFD08B10124A8
S315080041CC53E0FF20FFF74CFD10216846FFF7DBFD97
S315080041DC80B9012449E0FF20FFF742FD013DEDB20D
S315080041EC002DF8D19DF80A301A0910239340236044
S315080041FC00243AE03025F3E700210920FFF778FD83
S3150800420C08B1012431E010216846FFF7BCFD0028EF
S3150800421C7BD0434B1B6813F0020F11D09DF80A3064
S3150800422C5B0003F07E039DF80B2003EBD2130133DE
S3150800423C9DF80D209209013A93402360002414E05E
S3150800424C9DF80A30C3F384029DF80B10CB0003F0DB
S3150800425C180303EB5113013302FB033323600024C9
S3150800426C03E02F4B1B6813700024FFF71FFD2DE787
S3150800427C00210920FFF73CFD08B10124F5E71021C0
S3150800428C2046FFF780FD002841D10124EDE70021E7
S3150800429C0A20FFF72DFD08B10124E6E71021204678
S315080042ACFFF771FDA8BB0124DFE700213A20FFF7D1
S315080042BC1FFD054638B10124D7E7FF20FFF7D0FCD0
S315080042CC60550135EDB2032DF7D90024CDE7144B13
S315080042DC1B6813F0040F01D10124C6E700218D20B9
S315080042ECFFF706FD08B10124BFE7FF20FFF7B8FC6E
S315080042FC40212046FFF747FD68B90124B5E7042499
S3150800430CB3E70024B1E70124AFE70124ADE70024A5
S3150800431CABE70024A9E70024A7E700BF01000020AB
S3150800432C3411002000B583B000230193009303F1E8
S3150800433C804303F504331A6842F001021A6059687F
S3150800434C554A0A405A601A6822F0847222F480325E
S3150800435C1A601A6822F480221A605A6822F4FE023D
S3150800436C5A604FF41F029A601A6842F480321A6037
S3150800437C4A4B1B6803F400330093019B01330193EA
S3150800438C009B23B9019A40F2DC539A42F0D1434B75
S3150800439C1B6813F4003F79D0414B1A6842F010029F
S315080043AC1A601A6822F003021A601A6842F00202AE
S315080043BC1A60A3F580535A685A605A6842F4005238
S315080043CC5A605A6842F480625A605A6822F47C121F
S315080043DC5A605A6842F4E8125A601A6842F08072B7
S315080043EC1A602E4B1B6813F0007FFAD02B4B5A68B9
S315080043FC22F003025A605A6842F002025A60274BAE
S3150800440C5B6803F00C03082BF9D1244B9A6942F02C
S3150800441C09029A61234A516821F00F0151605168CB
S3150800442C41F008015160516821F0F0015160516862
S3150800443C41F0B0015160A2F54062516821F4C041C7
S3150800444C5160516841F480415160DA6942F000725A
S3150800445CDA61DA6942F40032DA619A6942F00502E5
S3150800446C9A61A3F584331A6822F470621A601A6882
S3150800447C42F430621A601A6822F470421A601A689A
S3150800448C42F480421A6003B05DF804FB6E210648BC
S3150800449CFCF782FB80E700BF0000FFF80010024023
S315080044AC00200240000C0140504D000808B5FFF7EB
S315080044BC39FFFCF7A9FBFCF7B7FBFCE7DFF834D0B0
S315080044CC002103E00C4B5B58435004310B480C4B52
S315080044DC42189A42F6D30B4A02E0002342F8043BF0
S315080044EC094B9A42F9D3FFF7E9F900F011F8FFF7EF
S315080044FCDDFF704700500020704E000800000020B9
S3150800450CD4010020D401002038110020FEE7000059
S3150800451C70B500250C4E0D4CA41BA410A54209D150
S3150800452C00F050F800250A4E0A4CA41BA410A5420C
S3150800453C05D170BD56F8253098470135EEE756F883
S3150800454C253098470135F2E7684E0008684E000892
S3150800455C684E00086C4E0008044B054A1B681B6A1B
S3150800456C002B08BF1346D3F8EC00704770010020E7
S3150800457C0400002082B001B901A942B14BB11378ED
S3150800458C0B601278101C18BF012002B07047104639
S3150800459CFBE76FF00100F8E703460244934200D1AB
S315080045AC704703F8011BF9E749B1FF2A8BBF8A2329
S315080045BC0A700360012088BF4FF0FF307047084629
S315080045CC70470000F8B500BFF8BC08BC9E4670479B
S311080045DCF8B500BFF8BC08BC9E46704746
S315080045E82E2E2F2E2E2F2E2E2F2E2E2F536F7572E0
S315080045F863652F41524D434D335F53544D3332460D
S31508004608312F63616E2E630005020602060307034F
S315080046180803090309040A040B040C040C050D0510
S315080046280E050F050F06100610071008006000088B
S315080046380020000003000000008000080020000099
S315080046480400000000A00008002000000500000083
S3150800465800C00008002000000600000000E000086E
S3150800466800200000070000000000010800200000E4
S3150800467808000000002001080020000009000000CA
S3150800468800400108002000000A0000000060010838
S31508004698002000000B000000008001080020000030
S315080046A80C00000000A00108002000000D00000012
S315080046B800C00108002000000E00000000E0010804
S315080046C8002000000F0000002E2E2F2E2E2F2E2E33
S315080046D82F2E2E2F536F757263652F41524D434DFA
S315080046E8335F53544D333246312F756172742E63D6
S315080046F800000000303A00002E2E2F2E2E2F2E2EC8
S315080047082F2E2E2F536F757263652F66696C652E6B
S31508004718630000004669726D77617265207570647A
S31508004728617465207265717565737420646574654E
S31508004738637465640A0D00004F70656E696E6720BC
S315080047486669726D776172652066696C6520666F41
S31508004758722072656164696E672E2E2E000000004D
S315080047684552524F520A0D004F4B0A0D00000000E1
S315080047785374617274696E67207468652070726F05
S315080047886772616D6D696E672073657175656E63AD
S31508004798650A0D0050617273696E67206669726DE5
S315080047A8776172652066696C6520746F2064657424
S315080047B865637420657261736520626C6F636B73D9
S315080047C82E2E2E0045726173696E67200000000060
S315080047D82062797465732066726F6D206D656D6FDA
S315080047E8727920617420307800000000526561648F
S315080047F8696E67206C696E652066726F6D206669DA
S315080048086C652E2E2E4552524F520A0D0000000096
S31508004818496E76616C696420636865636B73756D48
S3150800482820666F756E642E2E2E4552524F520A0D0B
S315080048380000000050726F6772616D6D696E6720BF
S315080048480000000020627974657320746F206D6516
S315080048586D6F727920617420307800005772697418
S31508004868696E672070726F6772616D206368656329
S315080048786B73756D2E2E2E00436C6F73696E6720E9
S315080048886669726D776172652066696C650A0D00DE
S315080048984669726D77617265207570646174652002
S315080048A87375636365737366756C6C7920636F6D6E
S315080048B8706C657465640A0D00000000809A4541AD
S315080048C88E418F804545454949498E8F9092924F2A
S315080048D8994F555559999A9B9C9D9E9F41494F5565
S315080048E8A5A5A6A7A8A9AAABACADAEAFB0B1B2B3F9
S315080048F8B4B5B6B7B8B9BABBBCBDBEBFC0C1C2C3EA
S31508004908C4C5C6C7C8C9CACBCCCDCECFD0D1D2D3D9
S31508004918D4D5D6D7D8D9DADBDCDDDEDFE0E1E2E3C9
S31508004928E4E5E6E7E8E9EAEBECEDEEEFF0F1F2F3B9
S31508004938F4F5F6F7F8F9FAFBFCFDFEFF010305079F
S31508004948090E10121416181C1E000000222A3A3CDA
S315080049583E3F7C7F000000002B2C3B3D5B5D000042
S31508004968C700FC00E900E200E400E000E500E70013
S31508004978EA00EB00E800EF00EE00EC00C400C50012
S31508004988C900E600C600F400F600F200FB00F900CC
S31508004998FF00D600DC00A200A300A500A72092010C
S315080049A8E100ED00F300FA00F100D100AA00BA0010
S315080049B8BF001023AC00BD00BC00A100AB00BB00C3
S315080049C891259225932502252425612562255625B4
S315080049D855256325512557255D255C255B25102515
S315080049E8142534252C251C2500253C255E255F2500
S315080049F85A25542569256625602550256C25672579
S31508004A0868256425652559255825522553256B2576
S31508004A186A2518250C25882584258C259025802522
S31508004A28B103DF009303C003A303C303B500C4039C
S31508004A38A6039803A903B4031E22C603B5032922AD
S31508004A486122B1006522642220232123F700482227
S31508004A58B0001922B7001A227F20B200A025A000AC
S31508004A6861001A03E0001703F8000703FF000100B6
S31508004A7878010001300132010601390110014A01A5
S31508004A882E017901060180014D0043028101820148
S31508004A9882018401840186018701870189018A01C7
S31508004AA88B018B018D018E018F0190019101910176
S31508004AB893019401F60196019701980198013D0220
S31508004AC89B019C019D0120029F01A001A001A20152
S31508004AD8A201A401A401A601A701A701A901AA0187
S31508004AE8AB01AC01AC01AE01AF01AF01B101B20136
S31508004AF8B301B301B501B501B701B801B801BA01E7
S31508004B08BB01BC01BC01BE01F701C001C101C2015C
S31508004B18C301C401C501C401C701C801C701CA0147
S31508004B28CB01CA01CD011001DD0101008E01DE01AC
S31508004B381201F3010300F101F401F401F801280157
S31508004B48220212013A020900652C3B023B023D0289
S31508004B58662C3F0240024102410246020A015302FC
S31508004B68400081018601550289018A0158028F0190
S31508004B785A0290015C025D025E025F0293016102BD
S31508004B886202940164026502660267029701960149
S31508004B986A02622C6C026D026E029C017002710236
S31508004BA89D01730274029F017602770278027902E0
S31508004BB87A027B027C02642C7E027F02A6018102AD
S31508004BC88202A9018402850286028702AE0144028E
S31508004BD8B101B20145028D028E028F02900291023E
S31508004BE8B7017B030300FD03FE03FF03AC030400C0
S31508004BF88603880389038A03B1031103C2030200E3
S31508004C08A303A303C4030803CC0303008C038E037E
S31508004C188F03D8031801F2030A00F903F303F40310
S31508004C28F503F603F703F703F903FA03FA0330045F
S31508004C38200350041007600422018A043601C104BF
S31508004C480E01CF040100C004D004440161052604FE
S31508004C58000000007D1D0100632C001E9601A01EA1
S31508004C685A01001F0806101F0606201F0806301FCF
S31508004C780806401F0606511F0700591F521F5B1FCB
S31508004C88541F5D1F561F5F1F601F0806701F0E0002
S31508004C98BA1FBB1FC81FC91FCA1FCB1FDA1FDB1FB6
S31508004CA8F81FF91FEA1FEB1FFA1FFB1F801F0806CC
S31508004CB8901F0806A01F0806B01F0400B81FB91FD2
S31508004CC8B21FBC1FCC1F0100C31FD01F0206E01F5E
S31508004CD80206E51F0100EC1FF21F0100FC1F4E210A
S31508004CE80100322170211002842101008321D02479
S31508004CF81A05302C2F04602C0201672C0601752C26
S31508004D080201802C6401002D260841FF1A030000C1
S31508004D184F70656E424C54002F626F6F746C6F67E4
S31508004D282E747874000000002F64656D6F70726FBA
S31508004D38675F6F6C696D65785F73746D3332703150
S31508004D4830332E73726563002E2E2F6D61696E2EB1
S31508004D58630000004300504F534958002E000020B6
S31508004D682020202020202020282828282820202005
S31508004D7820202020202020202020202020202088B5
S31508004D881010101010101010101010101010100419
S31508004D980404040404040404041010101010101069
S31508004DA8414141414141010101010101010101015D
S31508004DB80101010101010101010110101010101073
S31508004DC8424242424242020202020202020202022D
S31508004DD80202020202020202020210101010200049
S31508004DE800000000000000000000000000000000AD
S31508004DF8000000000000000000000000000000009D
S31508004E08000000000000000000000000000000008C
S31508004E18000000000000000000000000000000007C
S31508004E28000000000000000000000000000000006C
S31508004E38000000000000000000000000000000005C
S31508004E48000000000000000000000000000000004C
S31508004E58000000000000000000000000000000003C
S30908004E6831010008FE
S30908004E6C0D0100081E
S31508004E7004010000430000000000000000000000DC
S31508004E800000000000000000000000000000000014
S31508004E9000000000430000000000000000000000C1
S31508004EA000000000000000000000000000000000F4
S31508004EB000000000430000000000000000000000A1
S31508004EC000000000000000000000000000000000D4
S31508004ED00000000043000000000000000000000081
S31508004EE000000000000000000000000000000000B4
S31508004EF00000000043000000000000000000000061
S31508004F000000000000000000000000000000000093
S31508004F100000000043000000000000000000000040
S31508004F200000000000000000000000000000000073
S31508004F300000000043000000000000000000000020
S31508004F400000000000000000000000000000000053
S31508004F5000000000B5450008814500080000000073
S31508004F60664D0008644D0008654D0008654D00084B
S31508004F70654D0008654D0008654D0008654D00083B
S31508004F80654D0008654D0008654D0008FFFFFFFFE9
S31508004F90FFFFFFFFFFFFFFFFFFFF00000100415378
S31508004FA0434949000000000000000000000000001E
S31508004FB0000000000000000000000000000041534F
S31508004FC043494900000000000000000000000000FE
S31508004FD000000000000000000000000000000000C3
S31508004FE0740100200000000000000000000000001E
S31508004FF000000000000000000000000000000000A3
S315080050000000000000000000000000000000000092
S315080050100000000000000000000000000000000082
S315080050200000000000000000000000000000000072
S315080050300000000000000000000000000000000062
S30908005040000000005E
S705080044C9E5
